:1000000020C03AC039C038C037C036C035C034C04F
:1000100033C09BC731C030C02FC02EC02DC02CC0F4
:100020002BC02AC029C001020008200400000010D3
:1000300080401E0E1A2C32301224170713253B392C
:100040001B2D11241FBECFE5D4E0DEBFCDBF10E0D5
:10005000A0E6B0E0E2EBFBE102C005900D92A03615
:10006000B107D9F711E0A0E6B0E001C01D92A033BE
:10007000B107E1F7EBDA9CCDC3CF9FBB8EBBE09A13
:100080008DB3861719F06DBBE29AE19A0895FC01D1
:100090009085DF01A90FB11D8E918FB9779BFECF9F
:1000A0009150D1F7C19A1782C1980895DC014F731E
:1000B000FC01643010F033966450613061F06130BF
:1000C00028F06230C1F0633051F523C08081807C1C
:1000D000842B808324C080818F73942F9295990FF5
:1000E000990F907C982B90838181807F46954695CF
:1000F000842B818314C082818C7F942F92959F7072
:10010000892B828381818F704295407F482B418368
:1001100006C082818370440F440F482B428381E0E4
:10012000FD018783089587E09FEF9FB9779BFECFFE
:100130008150D9F797E01FB8779BFECF8FB1882306
:1001400019F485E090E008959150A9F787E090E0D8
:100150000895E82F772763FDEA5F86B323B330B3B2
:10016000482F41708695982F9270492B2470422B0E
:10017000869586958871307E832B482B64FD40954B
:10018000FF27EA5DFF4FE4914E23842F99270895BE
:100190008056904025E0959587952A95E1F708953A
:1001A00020E630E0F90180858D7F8087205E3F4F1B
:1001B000B09681E020323807B1F7089520E630E0AC
:1001C000E2E6F0E080819181B096009731F4205E04
:1001D0003F4F41E020323407A9F708951F93CF9392
:1001E000DF93DC01EC91EC0188858E2B84FD02C04D
:1001F0001FE306C0E295EF70FF27EE5CFF4F1491FE
:10020000CD01C6DF412F682F81E391E04FDFDF9101
:10021000CF911F910895FC018FEF868F908190619F
:100220009083808580FD61956295660F607E960F54
:100230009083CF01D3DF0895CF92DF92EF92FF92A8
:100240001F936B017C01122FBA01660F771F56FFB7
:1002500004C09B012250304003C09B012E5F3F4FE2
:10026000882777FD8095982F442737FD4095542F98
:1002700080DC05C0660F771F881F991F110F10348F
:10028000CCF320E030E0C616D706E806F90614F4F1
:1002900021E030E0C9011F91FF90EF90DF90CF90F7
:1002A0000895FC01828193810097B9F02481358102
:1002B00046815781AA2797FDA095BA2F820F931FD9
:1002C000A41FB51F632F691B84839583A683B783FF
:1002D000662319F06195CF019EDF0895CF93DF93D8
:1002E000C0E6D0E0CE01DDDFA09681E0C032D807C5
:1002F000C9F7DF91CF9108951F93CF93DF93EC015E
:100300001B8D46DFAC01212F332722FD07C08F85CF
:1003100087FD09C021FF09C088E01827612F842FBD
:1003200018DF992704C020FDF9CF8FEF90E0DF910F
:10033000CF911F910895FC0120E030E080819181F0
:10034000A281B38182509040A040B0488D5F9F4F02
:10035000AF4FBF4F10F421E030E0C90108951F9363
:10036000FC01138D10FF06C013DF612FF2DE282F72
:1003700033271CC08085992785FF03C020E030E02B
:1003800015C081FD02C060E00FC060E024813581AE
:100390004681578180899189A289B38928173907B5
:1003A0004A075B070CF461E0262F3327C9011F9130
:1003B00008951F93FC01838D81FF09C018E0182761
:1003C000CF01E6DE612FC5DE282F33271CC08085D4
:1003D000992785FF03C020E030E015C081FD02C0F1
:1003E00060E00FC060E024813581468157818489B7
:1003F0009589A689B78982179307A407B5070CF4D6
:1004000061E0262F3327C9011F910895FC01228541
:100410003385808183FF02C028E030E060FE08C0A1
:1004200080913A0190913B01821793070CF49C0153
:10043000C9010895FC01808182FF0BC082819381F4
:10044000813491051CF080858D7F80871382128214
:1004500014828081846080830895CF93DF93C0E607
:10046000D0E0CE01E7DFA09681E0C032D807C9F71F
:10047000DF91CF9108950F931F93CF93DF93EB01FB
:10048000042F122F85DE9C01E19918C080E390E0D3
:10049000A901489F9001499F300D589F300D1124AC
:1004A000285F3F4F200F311DFE013FBB2EBBE09A5E
:1004B0002F5F3F4F8DB381931150B9F7DF91CF91EB
:1004C0001F910F910895EF92FF920F931F93CF9377
:1004D000DF93EC01EC80FD800E811F81BC016C5F1D
:1004E0007F4F24E048E0C7DFBE01605F7F4F28E018
:1004F0004CE0CE01C0DF888587FF05C080E090E03A
:10050000A0E0B0E008C08C819D81AE81BF818E19D2
:100510009F09A00BB10B8C879D87AE87BF87DF91AA
:10052000CF911F910F91FF90EF900895FC0180856E
:1005300081FF37C014822089318942895389DA01C9
:10054000C90182509040A040B0488D5F9F4FAF4F8F
:10055000BF4F60F484819581A681B781281B390B38
:100560004A0B5B0B208B318B428B538B2489358953
:1005700046895789DA01C90182509040A040B048AD
:100580008D5F9F4FAF4FBF4F60F484819581A681EF
:10059000B781281B390B4A0B5B0B248B358B468BA1
:1005A000578B80858260808714821582168217821D
:1005B0000895CF93DF93C0E6D0E0CE01B7DFA096D9
:1005C00081E0C032D807C9F7DF91CF910895FC01CF
:1005D0008085992783FF03C0CF0175DF089582FFCF
:1005E00002C081E001C08FEF8787808182608083B5
:1005F0000895CF93DF93C0E6D0E0CE01E8DFA09668
:1006000081E0C032D807C9F7DF91CF910895EF920A
:10061000FF921F93CF93DF93CDB7DEB721970FB62D
:10062000F894DEBF0FBECDBF7C01FC01118519839C
:1006300021E045E0BE016F5F7F4F1DDF89811123FF
:1006400039F0882319F0811708F4182F80E406C0C8
:10065000182F8823D9F780E403C086951817E8F38C
:10066000F701818721960FB6F894DEBF0FBECDBF8C
:10067000DF91CF911F91FF90EF900895FC01808151
:10068000992783709070892B81F0818567FD09C05F
:10069000992787FD9095880F991F8187CF01B7DF34
:1006A0000895859519F081870895678F08950F93B0
:1006B0001F93CF93DF93CDB7DEB722970FB6F89491
:1006C000DEBF0FBECDBF8C0180E091E09A838983AD
:1006D00022E046E0BE016F5F7F4FC801CCDE89811A
:1006E0009A81009721F08F3F910519F014F080E076
:1006F00091E0F801228533852115310519F0821723
:10070000930718F4F8019387828722960FB6F8941E
:10071000DEBF0FBECDBFDF91CF911F910F91089526
:100720001F93CF93DF93EC01162F88819927837055
:100730009070892B91F0262F332727FD30958A85DD
:100740009B85280F391F2115310559F13B872A87D1
:1007500016163CF5CE01ABDF24C067FF05C0CE0105
:10076000FEDD882329F01DC0CE0123DE8823C9F4D5
:10077000212F332727FD3095322F2227442737FD9D
:100780004095542F8C819D81AE81BF81820F931F34
:10079000A41FB51F8C839D83AE83BF83612FCE01C1
:1007A0003ADDDF91CF911F9108950F931F938C0134
:1007B000BC016C5F7F4F2AE140E05DDEC80127DFAE
:1007C000C80175DF1F910F910895CF93DF93C0E6A5
:1007D000D0E0CE01EADFA09681E0C032D807C9F7A9
:1007E000DF91CF910895EF92FF920F931F93FC0139
:1007F000E088F188028913892489358946895789D7
:100800002E193F09400B510B203080E1380780E062
:10081000480780E05807F4F084819581A681B7816C
:100820008E199F09A00BB10B821B930BA40BB50B68
:100830000FB602FEF9CF820F931FA41FB51F0FB68C
:1008400000FEF9CF8E0D9F1DA01FB11F84839583DD
:10085000A683B7831F910F91FF90EF9008959F9209
:10086000AF92BF92CF92DF92EF92FF920F931F93BE
:10087000CF93DF93EC01B880AF8C0B2D1127C8010B
:1008800083709070892BA1F0F984FA0CFF8E00FD23
:1008900007C001FF05C0CE012FDD882311F076C10E
:1008A00080E002FD73C12FE32F150CF46FC190C1DE
:1008B00080E0CA80DB80988498012470307002FD4B
:1008C00044C001FF42C000FD40C0AF848F3F01F52E
:1008D0002C893D894E895F8988899989AA89BB8934
:1008E000A7FC09C02C873D874E875F878C839D833B
:1008F000AE83BF8308C08C879D87AE87BF872C835C
:100900003D834E835F8331E0B32A8DEF9822C8C0C8
:10091000882379F003FFC2C095EFB922CE01D3DD61
:1009200022E0922A14F431E0B32AAA24CC24DD2454
:10093000B7C08A2D992787FD90958C0D9D1D892B19
:1009400009F0AEC088E0B82AABC0C114D10409F4E4
:1009500075C0D7FE37C0232B29F4CE0100DD8823D4
:1009600009F416C194E0B92AD6C095FE0CC08C8556
:100970009D85AE85BF8581509040A040B04819F458
:10098000CE0131DF58C0EC80FD800E811F818C8547
:100990009D85AE85BF85E81AF90A0A0B1B0B2985D0
:1009A000A601C801B70148DC882329F50894C108CD
:1009B000D1082985A601C801B7013EDC882309F4C6
:1009C0006FC019C0232B29F4CE01F3DC882309F46E
:1009D000E2C034E0B32AFFEFAF2EA5C095FE0EC0F3
:1009E0008C859D85AE85BF858F5F9F4FAF4FBF477D
:1009F00029F4CE01F8DEE1E0AE2E52C0EC84FD8495
:100A00000E851F858C819D81AE81BF81E81AF90A10
:100A10000A0B1B0B2985A601C801B7010DDC882331
:100A200051F40894C11CD11C2985A601C801B70145
:100A300003DC8823A9F17FEFA72E32C0232B11F00E
:100A400034EFB322B0FE1EC02C853D854E855F85F8
:100A50008C819D81AE81BF81281739074A075B07CA
:100A60003CF4CE017CDC882359F46FEFA62E98C0AD
:100A70000FB601FC05C0CE019CDC882309F48EC0B2
:100A80008EEFB82293EFB922AA2051F48E8D8823DD
:100A900039F081508E8F882319F485C08EEFA826F7
:100AA000862D992780FF23C082FF08C020E0C03C2C
:100AB000D207E8F4888581FD7DC019C030E0C03CD4
:100AC000D30708F077C013C0CE0149DC882309F4AE
:100AD00076C051E0A52E0BC0CE016BDC882309F453
:100AE00071C04FEFA42E03C03FEFC32ED32ECE0113
:100AF0008DDC8C159D051CF42FEFA22E06C0C816A8
:100B0000D90619F41A140CF4AA24909581959F4FD4
:100B1000C816D9061CF481E0A82E05C0C816D9064F
:100B200011F4A7FCAA248A2D992787FD90958C0D96
:100B30009D1D2A81382F321B232F3985239F202D7D
:100B4000112429839B838A83892B91F48B2D9927E8
:100B500081FF0EC080FF0CC084EFB822CE01B3DC51
:100B600092E0992AB2FC04C097FE02C021E0B22AAA
:100B7000B8828B2D992783709070892B21F08F8DEF
:100B800080548F8F01C01F8E988622C0AA2491CED8
:100B900000FDEBCE85CF00FD21CF82CF01E0A02E5E
:100BA00033EFB3227DCF8FEEB822B882CE0116DBB1
:100BB0001C8276CF1C141D040CF48BCF85CFD7FE7E
:100BC0008BCF8FCF61FC90CF11E0C12ED12C8FCF76
:100BD000DF91CF911F910F91FF90EF90DF90CF9019
:100BE000BF90AF909F9008958091300181BFE0E069
:100BF000FEE009941F93CF93DF93162F60FE18C079
:100C000020913A0130913B01862F992787FD9095DD
:100C1000280F391F2115310509F457C081E0213013
:100C200038070CF052C030933B0120933A014DC07D
:100C3000882319F0CEE3D3E002C0C0E9D3E084E01A
:100C4000381641F1831560F081E03816C9F0381686
:100C500098F082E03816C1F083E03816B1F518C07C
:100C600086E0381629F13816C0F087E0381621F1F1
:100C700088E0381651F524C0612F80EC90E023C045
:100C8000612F80EE90E01FC0612F80E091E01BC0DB
:100C9000612F05C0612F619507C0612F619580EAC2
:100CA00090E0FE010995612F80E890E0FE01099532
:100CB000612F80E690E007C0612F80E890E003C0DC
:100CC000612F80EA90E0FE010995DF91CF911F919D
:100CD00008958C5D982F969596959695E92FFF2708
:100CE000EF5CFE4F877021E030E001C0220F8A9553
:100CF000EAF79081633011F492270CC0623011F44E
:100D0000922B08C0613021F4822F8095982302C075
:100D1000662321F0908381E0809338019223892F0C
:100D20009927089560E0882DD4DF882311F0A99ACF
:100D30000895A998089580912A01882341F081504F
:100D400080932A01882319F461E082E0C2DF0895CC
:100D50001F93182F682F882DBCDF112359F091E0C5
:100D6000891641F4882331F462E082E0B2DF8FEF2C
:100D700080932A01D7DF1F91089560FC6A946DDB90
:100D800008955D9B15C088E0681619F485E58CB957
:100D9000089590912D0180912C01981749F0E92F29
:100DA000FF27EC5BFD4F80818CB99F5F90932D01F5
:100DB0000895DC0130912C01262F932F8D91E92F7E
:100DC000FF27EC5BFD4F808321509F5F2223B1F70B
:100DD000360F30932C010895FF920F931F93CF93FA
:100DE000DF93082F803811F510913D01C0E0D0E06D
:100DF000EC2FFF27E45CFE4F8281E82FFF27A5E060
:100E0000EE0FFF1FAA95E1F7E05AFF4F8281938111
:100E1000892B41F0CF010EDB003819F40C2F00555F
:100E200001C00F6011502196112311F780912E01FE
:100E300090912F01891B87FF0BC080912C01E82F17
:100E4000FF27EC5BFD4F91E190838F5F80932C0136
:100E500080912C01E82FFF27EC5BFD4F00838F5F13
:100E600080932C018FE06822DF91CF911F910F9129
:100E7000FF9008951F93FC01162F828193810097A4
:100E800071F0181619062CF4CF0193DA882339F083
:100E900004C0CF0164DA882311F0812F9DDF1F91F8
:100EA0000895682F67FE13C080913D01681778F49C
:100EB000E62FFF27E45CFE4F82819927B5E0880F7B
:100EC000991FBA95E1F76053805A9F4FD3DF089579
:100ED0009927982F882780589040909329018093D4
:100EE0002801A89A089533B380B330953695369586
:100EF000369537708095880F8873382B832F992704
:100F000080729070892B11F080E13827222D207F8C
:100F1000832F9927807F9070821B9109880F991FDA
:100F2000880F991F859585953F70230F820F99270C
:100F30000895D9DF982F222D82258F70292E907F3A
:100F4000207F921B892B99270895189522B708B600
:100F500000FE02C02FEF06C080912001281710F478
:100F60002093200180912101821710F42093210108
:100F70008091220190912301AC01420F511D9A01F1
:100F800044275527542F432F322F2227AA27BB2728
:100F9000281B390B4A0B5B0B232F342F452F55276A
:100FA00047FD5A95309323012093220188B7882367
:100FB00029F478948895F89480E182BF81E088BF15
:100FC00080913801882319F081E391E060D886D9B7
:100FD00008950F931F93CF93DF93EC01142F022FEB
:100FE000242F3327402F5527C901840F951F819740
:100FF0000CF046C0CE01820F931FABD5010F1A3003
:1010000028F40A3028F0CE0102DB02C01C3020F4A4
:101010000B3010F0CE014BDB1C86013188F1888942
:101020009989AA89BB8982509040A040B0488D5FC1
:101030009F4FAF4FBF4F08F4188A8C899D89AE89A6
:10104000BF8982509040A040B0488D5F9F4FAF4F06
:10105000BF4F08F41C8A2C893D894E895F89888995
:101060009989AA89BB89281739074A075B0744F47D
:101070008C8B9D8BAE8BBF8B288B398B4A8B5B8B7C
:10108000DF91CF911F910F9108959F92AF92BF92E0
:10109000CF92DF92EF92FF920F931F93CF93DF9344
:1010A000CDB7DEB725970FB6F894DEBF0FBECDBF24
:1010B0008C017B01942E88E1841708F4A6C0442398
:1010C00009F4A3C0F801A484B584C684D784F1E0F0
:1010D000F41738F4242F21506F5F7F4F49E0C80187
:1010E00078DFF701E080ED82FF24E7FCF0948E2D9D
:1010F000807F09F08AC0C701877090700597E1F57D
:10110000F801808585FF02C0C8016DDBF8012485E8
:1011100035854685578529833A834B835C83808157
:1011200080FD04C0A480B580C680D7802A0D3B1DF9
:101130004C1D5D1D29833A834B835C830FB603FEF0
:1011400011C00FB602FE05C08FEF9FEFAFEFBFE7F4
:1011500004C081E090E0A0E0B0E889839A83AB838B
:10116000BC8301C0198289819A81AB81BC81F8015D
:1011700084879587A687B787E0FE27C0F80180851A
:1011800085FD23C0208931894289538984859585CD
:10119000A685B78582179307A407B50724F424878B
:1011A000358746875787F8012489358946895789C5
:1011B00084859585A685B785281739074A075B0773
:1011C00024F42487358746875787E1FE15C0F7E06A
:1011D000F91548F0F8018085FD818F278295880FE9
:1011E000807E805802C0F801878587FD02C081E0BB
:1011F00001C08FEFF8018787FD81FB7FFD83F80138
:101200008081FD818F2BF801808325960FB6F8949D
:10121000DEBF0FBECDBFDF91CF911F910F91FF9029
:10122000EF90DF90CF90BF90AF909F9008951F9365
:101230005F9BF2C13CB1462D4F7E642E45FF1BC023
:101240005C9B02C081EA0FC080912E01E82FFF272E
:10125000EC5BFE4F30838F5F80932E0190912F01C6
:10126000891719F482EAB8DDD7C1303809F0D4C142
:101270008FED6822D1C1252D552009F4C6C0E52D7A
:10128000FF27E45CFE4F30835394215080913D0151
:10129000281709F0C1C190913C01A92FBB27A77065
:1012A000B07065E0AA0FBB1F6A95E1F7A05ABF4F67
:1012B000892F8058863040F4293130F4422F6EE374
:1012C00071E0CD01E2DE9FC0892F8858863030F46E
:1012D000293120F448E06EE371E031C0892F8E5847
:1012E000823060F42150263008F08DC050E2652E27
:1012F000642A10922F0110922E0185C0892F8059E7
:10130000863090F4223081F480913E0160913F015B
:10131000282F3327C901860F911D819708F073C0CC
:10132000CD01820F931F3AC0892F8859863050F41F
:10133000223040F0215040913E016FE371E0CD0139
:1013400048DE61C0903A09F045C0243009F05BC026
:10135000E0913E01F0913F01809140016091410197
:10136000662309F450C087FD16C09F0150912C01DF
:10137000462F952FF9018491E92FFF27EC5BFD4F54
:1013800080832F5F3F4F41509F5F442399F7560F53
:1013900050932C0138C0803819F4CF010ADD33C0D6
:1013A000E19931C09F0140912C01562F942F3FBBF2
:1013B0002EBBE09A8DB3E92FFF27EC5BFD4F8083B6
:1013C0002F5F3F4F51509F5F552389F7460F409342
:1013D0002C0119C0913AB9F42430A8F080913E0153
:1013E00090913F0130914001303841F4422F552710
:1013F0004350504061E471E0ACD305C0313819F47A
:1014000083E080932B01552407C1832F81548630BC
:1014100050F4992745E0880F991F4A95E1F768E055
:10142000805A9F4F0FC0333241F480912C01E82F36
:10143000FF27EC5BFD4F3083E1C0343229F464E0D8
:1014400084E291E0B6DCE8C0353251F464E080E239
:1014500091E0AFDC8FEF8093200110922101DCC07E
:10146000363219F430E1632E7CC03F33B9F48091F9
:101470002C01E82FFF27EC5BFD4F93E590838F5FF6
:10148000E82FFF27EC5BFD4F9DE490838F5FE82FF3
:10149000FF27EC5BFD4F91E39083B0C0832F805317
:1014A000893010F4382EB8C0932F9754943150F4EB
:1014B00080913901873019F03B3408F0ADC0892E96
:1014C00031DCAAC03B3211F461E003C03D3221F4AB
:1014D0006FEF80E08FDBA0C0303401F510912C015C
:1014E000E12FFF27EC5BFD4F30821F5F882DE12F3E
:1014F000FF27EC5BFD4F80821F5F60E0EADBE12F9E
:10150000FF27EC5BFD4F80831F5FE12FFF27EC5B24
:10151000FD4F60821F5F10932C017EC0313619F49D
:1015200061E081E6D7CF323619F46FEF82E6D2CF91
:10153000333611F422DC70C0832F8451863058F486
:10154000832F992725E0880F991F2A95E1F780526C
:10155000924070D761C0343631F44095427081E0DA
:10156000682E642A59C0353629F44095427015E03A
:10157000612EF7CF373611F483E003C0383619F403
:1015800081E0E6DB49C0363611F413D845C0832F1D
:101590008E56863058F4832F9927B5E0880F991F0F
:1015A000BA95E1F780569D40C1D736C0343711F463
:1015B000F7D532C0832F8557863068F4E32FFF2795
:1015C000A5E0EE0FFF1FAA95E1F7E054FE408085ED
:1015D0008D7F808721C03E37A9F4F4E67F2E1092DC
:1015E00029011092280185B391E0892785BB80915C
:1015F0002C01E82FFF27EC5BFD4F20828F5F80934B
:101600002C010AC037FF08C030933C0110922B0117
:1016100047FD02C0E1E05E2E1F91089597DC07DED2
:1016200095DCAFDB08950F931F938C0149E050E0E8
:101630006FEF70E097D28FE0F801848315821682F5
:1016400072D5F80180871F910F910895FF920F9333
:101650001F93CF93DF9381B7809330019FEF91BFAA
:1016600022E023BF31E039BF80E885BF909320019D
:1016700085EF88BB8CE385BB8CEF82BB8AE287BB9E
:1016800083E084BB21BB80E58DB93EB981E391E065
:10169000CADF81E391E0FBD498D855247724442411
:1016A0006624332422241FDC282E80E490E09093CB
:1016B0003B0180933A0188E189B91BB88AB946DCBD
:1016C00080E690E0CCD85DDB41DC80E890E0C7D8D4
:1016D000AEDD3CDC80EA90E0C2D853DB37DC80EC46
:1016E00090E0BDD8A4DD32DC80EE90E0B8D849DBD4
:1016F0002DDC80E091E0B3D89ADD28DC1ADC77207D
:1017000009F07FC0C82FDD27CE018F719070892B23
:1017100009F477C0222D3327CE018223932383FF40
:1017200016C022FF0BC0862D962D9F5F9F70807F75
:10173000892B682E80FD0BC090D609C0832D8F5F4A
:10174000382E833008F03324832D8F5FC1DB222DA8
:101750003327CE018223932382FF2EC023FF15C09F
:1017600021E0821611F402E0802E982D9F5F892ED1
:1017700080913901853011F4943011F0943109F4DD
:101780008824D0DA882D8F5F16C0932D9F5F392E65
:101790008091680081FF03C022E030E002C025E0B4
:1017A00030E09350892F99272817390714F413E054
:1017B000312E832D82508CDBC1FDDFDA222D3327C1
:1017C000CE018223932380FF0EC0C901809590959E
:1017D0008F709070892B09F407DA21FF02C009D7B6
:1017E00002C083E0B5DAC4FF0CC0C5FF02C06FEFD2
:1017F00001C061E0641521F4822D8270FBD901C023
:10180000462E64FE14C080912B01882381F4D6D427
:10181000892B69F480912C01E82FFF27EC5BFD4FA9
:1018200096E290838F5F80932C013FEE6322A9DACA
:101830008DDB8091280190912901009769F0019733
:1018400090932901809328018F779070892B21F440
:1018500085B391E0892785BB6EDA872D772021F04B
:101860008150782E09F4A898E19942C0F0902B019C
:10187000FF20E1F000913E0110913F01EF2DFF2785
:10188000E45CFE4F6281C801F8D30F5F1F4F1093D5
:101890003F0100933E019F2D9F5F90932B0180910C
:1018A0003D01981729F510922B0122C0E0E6F0E0E7
:1018B00008E010E0808184FF04C0005D1F4FB096F7
:1018C00013C0EF012496FF246881C801D6D3E199A3
:1018D0000FC00F5F1F4F2196F39485E0F816A1F714
:1018E000055D1F4FFE01779621E0E032F20710F30D
:1018F0009EDC962D65FEE3CE80913C018295880F9B
:10190000880F807C682E692AB4E67B2E109229010C
:101910001092280185B391E0892785BB109224019C
:101920001092250110922601109227010CC176DE3B
:1019300080E0B7DA73DE81E0B4DA70DE82E0B1DA3B
:101940006DDE83E0AEDA6ADE84E0ABDA67DE85E086
:10195000A8DA64DEEEDA282F882379F090912C0142
:10196000E92FFF27EC5BFD4F2073822D8F70806481
:10197000822B80839F5F90932C0121FE02C080EA1E
:101980002BDAD9D94BDE262D67FEDDC010913D0143
:10199000F0902F0190912E019F1939F0EF2DFF2724
:1019A000EC5BFE4F8081803861F1911760F520E09B
:1019B00030E0E22FFF27E45CFE4FE281FF27A5E045
:1019C000EE0FFF1FAA95E1F7E05AFF4F8281938146
:1019D000892BE9F411502F5F3F4F112351F71EDE81
:1019E00080912E01992720912F01821B910920912E
:1019F0003D013327821793070CF0A5C0115079F7EA
:101A000081E8EAD9A0C097FF0DC093E10CC0822FF6
:101A10008054F7CF83EAF5CF802F8051F2CF802F0B
:101A20008052EFCF91E180912C01E82FFF27EC5BF2
:101A3000FD4F90838F5F80932C01C0E0D0E0A22FF8
:101A4000BB27A074B0700C2FEF2DFF27EC5BFE4F6F
:101A500090819038F9F2492F552747FD5095EC2F8A
:101A6000FF27E45CFE4F8281E82FFF2775E0EE0F31
:101A7000FF1F7A95E1F7E05AFF4F109739F199234C
:101A800009F446C0628173819A0157FF04C022277E
:101A90003327241B350B8185992787FD9095821765
:101AA00093070CF4B9CF9B01240F351FA90137FF11
:101AB00004C044275527421B530B82859385841706
:101AC00095070CF4ACCF3383228322C082819381AB
:101AD0009A01281B390BE1F037FF03C0309521959F
:101AE0003F4F8185992787FD9095821793070CF4C6
:101AF00093CF9A0157FF04C022273327241B350BAD
:101B000082859385821793070CF489CF5383428390
:101B1000F39411502196112309F095CF809124015F
:101B200090912501A0912601B09127010196A11D58
:101B3000B11D8093240190932501A0932601B093B9
:101B40002701F0922F0167FCF2CE17D97724A898CD
:101B5000B6CDFB01DC0102C001900D924150504016
:101B6000D8F70895DC0101C06D9341505040E0F773
:101B70000895629FD001739FF001829FE00DF11DD7
:101B8000649FE00DF11D929FF00D839FF00D749FF7
:101B9000F00D659FF00D9927729FB00DE11DF91FA3
:101BA000639FB00DE11DF91FBD01CF011124089500
:021BB000FFCF65
:00000001FF
